:0404000002048D3233
:01040B0032BE
:0104130032B6
:01041B0032AE
:0104230032A6
:01042B00329E
:010433003296
:01043B00328E
:010443003286
:01044B00327E
:010453003276
:01045B00326E
:0304630002161F5F
:01046B00325E
:010473003256
:01047B00324E
:03048300020A6208
:0704E600E4F508F509E4F557
:0404ED000AF50B7889
:0504F10000E4F208F236
:03053C0002048630
:050486001205C480FE18
:03053F0002177828
:09054200AA82E5082443F582E5D4
:08054B000934F0F583EAF00524
:0605530008E4B5080205F2
:010559000998
:01055A00227E
:06055B00E4F50AF50BE5D2
:06056100084509605D126F
:080567000E68AA82E508C395A5
:05056F000AFBE50995FF
:0C0574000BFC8A057E00C3EB9DEC9E5042
:080580001FE50A2443F582E5A2
:060588000B34F0F583AB1B
:07058E0008AC0AEBC39C78E6
:0705950010F2120E9CE4F5C8
:04059C0008F5092233
:0705A000E50A2443F582E5A2
:0605A7000B34F0F583782F
:0C05AD0010EAF2C002120E9CD0027B008B
:0705B900EA250AF50AEB3503
:0305C0000BF50B2D
:0105C3002215
:0705C400121557120F23125C
:0205CB000731F6
:0905CD00120778400B12156312AD
:0705D6000DCF43FF0280F08E
:0305DD0053FFFDCC
:0705E000120DCF121563128A
:0C05E7000806E5828583F07800F208E544
:0C05F300F0F212053F7800E2F5F008E29B
:0C05FF0045F060DD63FF027800E2F58249
:0E060B0008E2F583E0FAC002120826AB82D0A6
:0B06190002BB0260C00274A7C0E074C6
:0C0624001FC0E07480C0E012182815818F
:0806300015811581D0027C0048
:04063800ECB502001B
:05063C00400302071B52
:090641008C057E000DBD00010EC8
:0C064A007800E22DF58208E23EF583E026
:0C065600FD7E00C002C004C005C0067498
:0A066200B4C0E0741FC0E07480C053
:0E066C00E0121828E58124FBF581D004D002AD
:03067A000C80BB36
:05067D00BB0102800337
:0306820002071B51
:0A06850074BAC0E0741FC0E0748076
:0C068F00C0E01218281581158115817833
:0C069B0000E22401F58208E23400F5833F
:0C06A700E0FAA3E0FBC002C00374C7C06F
:0C06B300E0741FC0E07480C0E012182842
:0C06BF00E58124FBF5817800E22403F5BE
:0E06CB008208E23400F583E0FAA3E0FBC002EF
:0A06D900C00374D8C0E0741FC0E035
:0E06E3007480C0E0121828E58124FBF58178B0
:0C06F10000E22405F58208E23400F583E5
:0C06FD00E0FAA3E0FBC002C00374E9C0F7
:0C070900E0741FC0E07480C0E0121828EB
:06071500E58124FBF581E3
:06071B001208397810E518
:0607210008F290F0431203
:060727000E9CE4F508F54C
:04072D00090205E0D8
:0D1FA70043414E204D4553534147450A002C
:061FB400307825780A00D8
:0D1FBA00494D55204D4553534147450A0000
:0E1FC700616363656C58206973203A202564BD
:031FD500200A00DF
:0E1FD800616363656C59206973203A202564AB
:031FE600200A00CE
:0E1FE900616363656C5A206973203A20256499
:031FF700200A00BD
:0704F600750C00750D007587
:0604FD000E00750F0075F2
:050503001000C200C25F
:0105080001F1
:06073100121F79D203C281
:0C0737000490DF027413F0901FFAE493AA
:0E074300FA74019374029374039390DF06EA34
:07075100F0D201120B85D26A
:0407580000020B7F11
:05075C0074C8B5100097
:0607610050047AFA800248
:020767007A0115
:0E076900C002120C46E582D00254032AF5822B
:01077700225F
:04077800A200B32206
:0A077C00E50FC3950E14540FF5822B
:010786002250
:0A078700E50EC3950F540FF5822212
:0B07910012077CE5827004900000223B
:0A079C00E50E75F014A424DDFA74D4
:0907A600F235F0FB0ABA00010B68
:0507AF008A828B832209
:0A07B400AA82E50E75F014A424DDFE
:0A07BE00FB74F235F0FCE50E75F057
:0A07C80014A424DDFD74F235F0FEE8
:0E07D2008D828E83A3E0FD0D8B828C83EDF073
:0A07E000E50E75F014A424DDFB748F
:0C07EA00F235F0FC8B828C83A3EA2AFA23
:0A07F600F0740FB50E05750E0080BB
:0108000002F5
:02080100050EE2
:03080300020B7F66
:09080600E50DB50C049000002280
:0A080F00E50C75F016A4249BFAE432
:0808190034F2FB0ABA00010BE6
:050821008A828B832296
:0A082600E50C75F016A4249BF58282
:09083000E434F2F583E0F58222C4
:090839007402B50C04750C0022D8
:03084200050C2280
:0D08450090F41D7401F090F41E74C0F0904A
:08085200F41D120C07740125CE
:05085A00104002051032
:01085F002276
:0A086000AA82E50F75F014A424DD50
:0B086A00FB74F235F0FC0BBB00010C2E
:0A087500E50F75F014A424DDFD74F6
:0C087F00F235F0FE8D828E83A3E0541E43
:0C088B004202A204E43342028B828C8300
:0A089700EAF0E50F75F014A424DD6B
:0B08A100FA74F235F0FB8A828B8312A0
:0908AC000C07740125104002053F
:0108B5001032
:0108B600221F
:0708B700300006120845D2D3
:0208BE00052211
:0708C000E50EB50F028009EF
:0908C700758200120860D20522BE
:0A08D000E50D75F016A4249BFAE470
:0A08DA0034F2FB7808E4F28A828B06
:0408E40083020BA9D7
:0808E800AA82BA21030208B73D
:0A08F000BA1E25E50D75F016A424CC
:0A08FA009BFBE434F2FCC003C004D1
:0C09040012075CAD82D004D0037808ED2F
:08091000F28B828C83020BA91B
:05091800BA1F0280037C
:03091D00020A5B70
:09092000E50D75F016A47806241B
:080929009BF2E434F208F21223
:07093100174A402CE50EB54A
:040938000F02801515
:0A093C0012075CAD827808EDF27836
:0B09460006E2F58208E2F583020BA92F
:0A0951007808E4F27806E2F5820867
:06095B00E2F583020BA986
:0C0961007806E22401FD08E23400FE8D5F
:0D096D00828E83E0FF74C05FFBBBC019D217
:04097A0003D2029012
:0C097E00F41D7401F090F41E7480F090E1
:06098A00F41D120C07D25F
:0209900005223E
:0D099200C005C00674C05FFDBD8002800678
:06099F00D006D0058028FF
:0909A500D006D005100002800705
:0709AE00751000C20480185F
:0709B500E50EB50F028011F1
:0A09BC00740FB50F05750F008002DF
:0209C600050F1B
:0509C800751000B204EF
:0B09CD007806E2F58208E2F583E0F511
:0609D800117401B51100CD
:0C09DE0050787B80200114C00374015F7E
:0C09EA00FCA203E433FBB50404D003803E
:0109F6003FC1
:0209F700D0032B
:0909F9007402B50D047C008004B9
:040A0200E50D04FCFE
:060A0600ECB50C02802893
:0A0A0C00C003EF139203C201530769
:0C0A16001EEFC313FFE511148D828E83C8
:0C0A2200F07806E2F58208E2F583EFF0C0
:060A2E008C0DD0038002D4
:020A34007B4005
:070A3600E50EB50F02800779
:070A3D008B8212086080119A
:0C0A440090F41D7401F090F41EEBF09093
:050A5000F41D120C076B
:030A5500D20522A5
:030A58000208B7DA
:060A5B00BA20030208B7F7
:010A61002272
:041FFA008000000063
:06050900751200C206C2DB
:03050F0007C20818
:0C0A6200C024C0E0C0F0C082C083C0020D
:0E0A6E00C003C004C005C006C007C000C00120
:0E0A7C00C0D0E4F5D0F59BE5E930E418740332
:0B0A8A00B5120875821E120B21800BB4
:0B0A95007402B5120675821F120B21BF
:0B0AA000E5E930E506758220120B210D
:0A0AAB003006427403B51202804FBA
:0C0AB5007402B5122390DF3BE0FABA0D8A
:0E0AC1001B90DF3CE0FA20E33A90DF12E0FAEF
:080ACF00530207BA070280067A
:060AD70074F625A450276F
:0A0ADD0090DF3BE0FABA0D0280033F
:030AE70075E104B2
:060AEA00758221120B21B0
:0A0AF000E5E930E705D20875E97F5B
:0A0AFA00E5E930E605D20775E9BF13
:0E0B0400D0D0D001D000D007D006D005D0044C
:0D0B1200D003D002D083D082D0F0D0E0D04C
:020B1F0024327E
:0C0B2100AA8290DF3BE0FBBB1202801EAA
:0A0B2D0090DF3BE0FBBB01028014E7
:0E0B370090DF3BE0FB600D90DF3BE0FBBB1569
:030B450002800328
:030B480075E10054
:0C0B4B0075D68253D1FD75120290DF12A6
:0C0B57007407F08A821208E875E9CFAA42
:060B630012BA0202800537
:050B6900BA0310800832
:080B6E0043D60275E102800686
:060B760043D60275E10305
:030B7C00C206228C
:060B7F00D206439B032295
:0E0B85001216AB90DF147414F090DF13740599
:0E0B9300F090DF127407F0439A017591F0D2D2
:080BA100AF90F4327413F0224E
:0C0BA900AA82AB837808E2601290DF1291
:0C0BB500E4F075A2007808E2F5A475A336
:030BC100008006AB
:060BC40090DF127407F03F
:0E0BCA007CD97D0074DF2DFC90F42CECF07CC7
:0E0BD800D990F42DECF08B0490F42EECF090FC
:0D0BE600F42FEAF090DF02E0FA0A0A0A900C
:0B0BF300F431EAF090F4307480F090D0
:090BFE00F4337410F075120222A8
:0E0C0700AA82AB838B0490F42CECF090F42DB9
:0E0C1500EAF07AD97B0074DF2BFA90F42EEA15
:0E0C2300F07AD990F42FEAF090DF02E0FA0A9E
:0C0C310090F431EAF090F4307420F09060
:090C3D00F4337440F07512032237
:0604BC00E478FFF6D8FD14
:080C4600E5B4540C600280F8D3
:0C0C4E0085BC82743055B44407F5B42214
:0A0C5A00AA827809E27003EA60093B
:090C64007809E2B40308BA800526
:050C6D00780974AAF2F1
:0B0C72008ABC7809E2F5BC120C4612A7
:050C7D000C46020C46CC
:08049A007909E94400601B7AB6
:0504A2000190209D788F
:0304A7004C7593FE
:0A04AA00F4E493F2A308B800020581
:0804B40093D9F4DAF27593FF0D
:06051200751300C209C2CE
:060518000A780AE4F27803
:09051E000BE4F2780C74FFF27A90
:04052700077B0D78C9
:06052B000DEAF208EBF2FC
:0C0C8200781D740AF27582011214F378D8
:0B0C8E001E7440F275820412152578D8
:0B0C99001D7440F27582041214F37801
:050CA4000C74FFF222B8
:0E0CA90090F420E0FA53027FBA215190F42417
:0E0CB700E0FAA3E0FB4A6006BA0143BB00402E
:0A0CC50090F421E0FABA2002800A40
:050CCF00BA21028014AF
:050CD400BA222E801E73
:070CD900781B744CF2087453
:080CE000F4F29000070214BEBB
:070CE8007819744CF2087446
:080CEF00F4F290000702149DCD
:0C0CF70090F422E0FAA3E0780AEAF2028E
:020D030014DFFB
:010D050022CB
:010D060022CA
:010D070022C9
:0C0D0800780DE2F58208E2F58312048BFE
:0E0D140090F44CE0FAA3E0FBA3E0FCA3E0FDAA
:0D0D2200BA4D1DBB011ABC0017BD00142006
:050D2F000A11D20A12B6
:0E0D34001644AA82AB83ACF0FD90F41FEAF0E7
:010D4200228E
:0A0D430090F453E0FABA10028004A5
:040D4D007582002289
:0E0D510090DE0E7404F090DE14E0FA30E0073D
:070D5F0090DE16E0F5822290
:040D66007582002270
:0E0D6A0090DE0E7404F090DE28E0FA90DE16A3
:0C0D7800E0FB700890DE14E0FB54FEF07D
:050D8400D20C8A82225E
:0A0D8900AA82AB83780F7913E2F31E
:0B0D93007814EAF208EBF275820412FB
:0E0D9E000F2490DE16E0FA700890DE14E0FAE2
:030DAC0054FEF002
:010DAF002221
:0E0DB00090DE0E7404F090DE11E0FA4401F0C3
:080DBE007440B51303D380015A
:010DC600C369
:060DC7009209751300D231
:020DCD000C22F6
:070DCF00120F9C300A1B12F9
:0E0DD6001644AA82ACF0FD90F41FE0FBEAC3C5
:070DE4009BFA7446B5020002
:050DEB0050031215D3B6
:0A0DF00090F453E0FABA10028001FB
:010DFA0022D6
:0B0DFB0090DE0E7404F0E513700B3066
:0A0E0600090B90DE11E0FA20E10371
:030E1000120DB010
:0A0E130090DE0E7401F0780B790CEC
:080E1D00E2F5F0E3B5F001225B
:0E0E250090DE11E0FA20E03A90DE2274A1F097
:0E0E33007420F0E4F0E4F090DE22F0E4F074BD
:0C0E410002F0E4F0780B90DE22E2F0906A
:0C0E4D00DE22E4F090DE11E04401F078B9
:0A0E59000BE25483F2780BE2FA7802
:040E63000CF2D20CAF
:010E67002268
:0A0E680090F453E0FABA100280047F
:040E72007582002263
:0E0E760090DE0E7404F090DE11E0FA30E11010
:080E8400EA30E004758200224F
:080E8C007440C39513F58222A6
:080E94007480C39513F582225E
:040E9C00AA82AB83F8
:0A0EA0007810E260527440C395130D
:070EAA00FC7810E2B5040022
:060EB10050047810E2FC81
:0A0EB7007816ECF27817EAF208EB67
:0E0EC100F2758204C002C003C004120F59D0A3
:0C0ECF0004D003D002EC2AFAE43BFB78CC
:090EDB0010E2C39CF2EC2513F5B2
:0A0EE400137440B513B6C002C0033A
:090EEE00120DB0D003D00280A95E
:010EF70022D8
:0B0EF800E58290DE28F005137440B581
:050F03001303020DB014
:010F080022C6
:060F0900780AE2F58222E5
:0A0F0F00AA82780BE2547C4A780BAA
:020F1900F222C2
:080F1B00AA82780BE24AF222DF
:0E1FFE001201000202000020FB1F0022000062
:04200C0001020301C9
:0E20100009024300020100C032090400000171
:0E201E00020201000524002001042402020534
:0E202C00240600010524010001070581030AB6
:0E203A00000109040100020A0000000705046D
:0B204800024000000705840240000079
:012053000488
:042054000403090474
:0E205800260350006F006C006F006C007500D6
:0E206600200043006F00720070006F007200D7
:0A2074006100740069006F006E0047
:0C207E000C0357006900780065006C003E
:02208A005420E0
:02208C005820DA
:02208E007E20B2
:02209000E60365
:07209D00802500000000088F
:04053100C20BC20C2B
:010F230022AB
:0E0F2400AA82E4CA25E0CA33FB74202AFA74BC
:0A0F3200DE3BFB7813E2FC7814E2CA
:040F3C00FD08E2FECC
:0E0F4000EC60131C8A828B83E0FF8D828E830F
:080F4E00F0A3AD82AE8380EA3E
:030F5600D20C2298
:0E0F5900AA82E4CA25E0CA33FB74202AFA7487
:0A0F6700DE3BFB7816E2FC7817E28F
:040F7100FD08E2FE97
:0E0F7500EC60141C8D828E83E0FFA3AD82AE73
:090F8300838A828B83EFF080E980
:010F8C002242
:0C0F8D00C20B90DE017401F090DE0B74CA
:030F990007F0223C
:0C0F9C0012160C400E53BE7F121615906A
:070FA800F453E4F0C20B2238
:0E0FAF0090F453E0FA701312161943BE80003E
:0C0FBD0000000090F4537402F0120F8D3D
:0E0FC90090DE06E0FA90DE02E0FBEA30E00285
:020FD700D20B3B
:0E0FD900EA30E21690F4537404F090F454E4FD
:0C0FE700F0C002C003120F8DD003D00236
:060FF300EA30E102C20B2E
:050FF900EB20E00122E5
:0C0FFE0090DE0EE4F090DE11E0FAD20C60
:0E100A00EA30E40B90DE117480F090F454E4B0
:01101800F0E7
:0D101900EA30E20990DE11E4F090F454F0AA
:07102600EA20E00302114F74
:0A102D0090F454E0FBBB01028003C5
:031037000210D5CF
:0E103A0090DE16E0FB90F428E0FCA3E0FD8BB6
:0C104800067F00C3EC9EED9F50028C035D
:071054007813EBF27811792B
:0C105B0014E2F308E209F3758200C00201
:0C106700C003120F24D003D0027811E265
:0E1073002BF208E23400F27C0090F428E0FD3D
:0E108100A3E0FE90F428EDC39BF0EE9CA3F0DC
:0E108F0090F428E0FBA3E0FC4B600990DE111A
:06109D007440F002114F47
:0E10A30090F420E054606007C002120D08D0E7
:0110B100023C
:0D10B20090DE0EE4F090F454E0FB70099025
:0810BF00DE117468F002114F0C
:0E10C70090DE117448F090F454E4F002114FE2
:0C10D50090DE16E0FBBB086C781374087A
:0810E100F278147420F2087487
:0C10E900F4F2758200C002120F24D00245
:0E10F50090F454E4F090F420E054607009C0D0
:08110300021211BAD0028007AC
:07110B00C002120CA9D00282
:0D11120090DE0EE4F090F454E0FB700890C5
:07111F00DE117460F080296D
:0E112600BB012690F428E0FBA3E0FC4B600820
:0811340090DE117440F08013FD
:0D113C0090DE11744AF090F454E4F0800647
:0611490090DE117440F07D
:0D114F00EA20E16690F454E0FBBB025E90E4
:0E115C00F428E0FBA3E0FCC3EB9420EC94002D
:0B116A0050097A0A90F454E4F080046D
:041175007A027B205F
:071179007816EBF278117902
:0C11800017E2F308E209F3758200C002D8
:0E118C00C003120F59D003D00290DE11EAF01A
:0C119A007811E22BF208E23400F27A0037
:0E11A60090F428E0FCA3E0FD90F428ECC39B3D
:0511B400F0ED9AA3F02C
:0111B9002213
:0A11BA0090F42AE4F090F42BF0907A
:0911C400F421E0FA740CB50200FC
:0311CD00500122AC
:0711D000EA2A2A9011D773EF
:0711D7000213830214380229
:0611DE00144A021438025D
:0611E400144A0212CD02C4
:0611EA0011FE02144A028E
:0611F00013260212EB02BF
:0611F600134802144A0236
:0211FC00143BA2
:0E11FE0090F422E0FAA3E0FBFC7D00BC0105AA
:05120C00BD000280138B
:08121100BC0205BD00028020B3
:08121900BC0305BD0002803991
:0312210002129C1A
:07122400781174FEF208745A
:0C122B001FF290F4287412F0A3E4F0020B
:0212370012A7FC
:04123900EA60012244
:07123D0078117410F208742F
:0C12440020F2902012E493FCA3E493FD40
:0A12500090F428ECF0A3EDF0804DBF
:0E125A008A047D00902053E493FE7F00C3ECD5
:061268009EED9F400122F3
:0C126E00E4CA25E0CA33FBEA248AF582BA
:0C127A00EB3420F583E493FAA3E493FB2B
:0C1286007811EAF208EBF28A828B83E018
:0A129200FA90F428F0A3E4F0800BBA
:0B129C00120D0690F454E0FA700122DD
:0E12A70090F426E0FAA3E0FB90F428E0FCA30C
:0E12B500E0FDC3EA9CEB9D500890F428EAF09F
:0312C300A3EBF0AA
:0712C60090F4547402F022C1
:0E12CD0090F422E0FAA3E0FB90DE00EAF0EAE3
:0612DB0060047A088002A5
:0212E1007A048D
:0812E30090F453EAF00214DF5D
:0E12EB0090F422E0FAA3E0FBBA0005BB00027B
:0212F90080086B
:0812FB00BA0124BB002180149C
:0A13030090F453E0FA7408B50200FC
:0A130D00501490F4537408F0800CA3
:0B13170090F4537410F0120C8280015F
:0113220022A8
:031323000214DFD2
:0C13260090F453E0FABA10047A0180023F
:021332007A003F
:0813340090F42AEAF078197424
:0A133C002AF20874F4F29000010296
:02134600149DF4
:0813480090F453E0FABA100022
:0313500050012227
:0B13530090F424E0FAA3E0FB7C107D86
:0C135E00208C828D83A3A3A3A3E493FC46
:0A136A007D00C3EA9CEB9D400122C8
:071374007819742AF20874D5
:08137B00F4F290000102149D40
:0E13830090F420E0541FFA7B00BA0005BB0076
:03139100028014C3
:08139400BA0105BB0002802B29
:09139C00BA0206BB000302140DA5
:0313A500021437F8
:0913A80012161250047A018002B1
:0213B1007A00C0
:0813B30090F42AEAF0781974A5
:0A13BB002AF20874F4F29000020216
:0213C500149D75
:0813C70090F453E0FABA1000A3
:0E13CF00500C90F424E0FAA3E0FB4A600122E7
:0B13DD0090F424E0FAA3E0FB7C107DFC
:0C13E800208C828D83A3A3A3A3E493FCBC
:0A13F4007D00C3EA9CEB9D4001223E
:0713FE007819742AF208744B
:08140500F4F290000202149DB4
:0E140D0090F422E0FAA3E0FBEA540F600280A4
:01141B0001CF
:01141C0022AD
:08141D0090F453E0FABA10004C
:0314250050012251
:071428007819742AF2087420
:08142F00F4F290000202149D8A
:011437002292
:031438000214DFBC
:07143B007819742AF208740D
:08144200F4F290000212149D67
:01144A00227F
:03144B00A20B22CF
:0C144E00AA8CA2BD920DC2BD438C1053AD
:02145A008CFE06
:0E145C00758900C2C5D2BDABBE74FC5B4401F5
:0E146A00F5BE000000E5BE54036007D29043BB
:041478008701C29096
:09147C00C2BDE58930E702C20B94
:0C148500300B09C002121612D00250CB2E
:0C149100E5BE30E6FB8A8CA20D92BD2265
:0E149D00AA82AB8390F4547402F090F428EA13
:0C14AB00F0A3EBF07819E2FA08E2FB78FD
:0714B70011EAF208EBF2223A
:0E14BE00AA82AB8390F4547401F090F428EAF3
:0C14CC00F0A3EBF0781BE2FA08E2FB78DA
:0714D80011EAF208EBF22219
:0E14DF0090F4547401F090F428E4F0A3F0228D
:0614ED0090F454E4F0222B
:0C14F300E58290DE0EF0781DE2FA7B002E
:0E14FF0074072AFAE43BFBC423CAC423541F1B
:0C150D006ACA541FCA6ACA30E40244E0F3
:0C15190090DE10EAF090DE127401F02267
:0C152500E58290DE0EF0781EE2FA7B00FA
:0E15310074072AFAE43BFBC423CAC423541FE8
:0C153F006ACA541FCA6ACA30E40244E0C1
:0C154B0090DE13EAF090DE157401F0222F
:0120A400003B
:0120A500003A
:05053500781F7480F244
:07155700121578121566124F
:05155E0016650216A451
:031563000215FA74
:0315660053BEFB76
:0E156900E5BE30E6FB75C68043BE0475C700C4
:011577002251
:0A15780075FF0075A00675F79922B3
:0C158200121644AA82AB83ACF0FD781F67
:0A158E00D3E29AF4FA7419B50200D2
:0C1598005038E5FFA2E4920F400943FF29
:0715A40010758202121F9F67
:0E15AB0053F7EF53FFEF758201121F9FA2A4AA
:0A15B900920E43F710300F0343FFBA
:0115C3001017
:0C15C400121644AA82AB83ACF0FD781F25
:0215D000EAF23D
:0115D20022F6
:0E15D300C2AF75D69F75820A121F9F75FF006A
:0E15E10075FE0075FD0075F50075F40075F3DC
:0B15EF0000900064121670020006223B
:0E15FA00E5FF20E20C75820A121F9F30A2034B
:031608000215D3F5
:01160B0022BC
:06160C00121582A20E225D
:03161200A2A3226E
:0416150053FFFE225F
:06161900D2A043FF0122F4
:0C161F00C0E0C000C0D075D0007820E210
:0E162B002401F208E23400F208E23400F20872
:0B163900E23400F2D0D0D000D0E0324C
:0C164400A2BCE433FAC2BC7820E2FB0830
:0E165000E2FC08E2FD08E2FEEA24FF92BC8BF9
:07165E00828C838DF0EE2267
:0B16650075EDBBD2BC75EBFAD2AF22D2
:04167000AA82AB831C
:091674008A048B051ABAFF011B60
:0E167D00EC4D60227582FAC002C003121F9F5E
:0E168B007582FA121F9F7582FA121F9F7582D8
:0A169900F9121F9FD003D00280D188
:0116A3002224
:0804C2007843E84400600A7968
:0304CA0000759327
:0604CD00F0E4F309D8FC85
:0804D3007809E84404600C798B
:0B04DB000590F000E4F0A3D8FCD9FA73
:0716A40075D22C75D3F4226E
:0D16AB0090DF2E74FEF090DF097464F09063
:0E16B800DF0A7425F090DF0BE4F090DF0F7472
:0E16C60043F090DF107487F090DF07740AF095
:0E16D40090DF08E4F090DF0C741DF090DF0D45
:0E16E20074DEF090DF0E7473F090DF1A74B6B1
:0E16F000F090DF1B7410F090DF15741DF09069
:0E16FE00DF16741CF090DF1774C7F090DF1831
:0E170C00E4F090DF1974B2F090DF1C74EAF084
:0E171A0090DF1D740AF090DF1EE4F090DF1FD8
:0E1728007411F090DF237488F090DF24743188
:0E173600F090DF257409F090DF037404F0904A
:06174400DF047445F022F1
:06174A0090DF39E03322BC
:0B17500090DF39E0FA747F5AF5822226
:0E175B0090DF3AE0FAC2D575F002EA30E704FA
:04176900B2D5F404FD
:06176D008430D502F404F3
:0517730024B9F58222FB
:02048B00E47318
:02053A00C210ED
:05177800100C028015B9
:0A177D0090DE0CE0FA7824F2201050
:0A1787000AD21090DE0CE0FA78257B
:01179100F265
:0C17920012144B400790F453E0FA70046E
:04179E0053FFEF22E4
:0C17A200BA103D30103690DE0CE0FA7BEF
:0C17AE00007825E2FC7D00EAC39CFAEB09
:0B17BA009DFBEA30E60543FF108003B2
:0317C50053FFEFE0
:0C17C80090DE0CE0FA7824D3E29AF4FAE8
:0517D4007460B5020085
:0517D900501DC21022AA
:0417DE0043FF102293
:0E17E200121644AB83ACF0FDEB035401FA6029
:0517F0000443FF10227C
:0317F50053FFEFB0
:0117F80022CE
:0617F900C01885811812E2
:0517FF000542D0182294
:0C180400AA82AB83ACF07833E4F208F267
:0C18100008F27836EAF208EBF208ECF27D
:07181C0078267939E2F39010
:0518230017F902191E77
:06182800C018858118E5DF
:0A182E001824FBFA7833E4F208F204
:0A18380008F2E51824FBF87936E603
:0C184200F30809E6F30809E6F37839EA38
:08184E00F29017F912191ED0E7
:02185600182256
:0C185800AA827829E2C0E008E2C0E008A3
:0A186400E2C0E0747BC0E07418C01D
:0C186E00E07827E2C0E008E2C0E08A82D7
:01187A00224B
:0C187B001581158115817831E22401F2FD
:0618870008E23400F22229
:0B188D00AA8274302AFA7439B50200F8
:0C189800500A74072AFA301103430220A2
:0518A4008A82021858C1
:0E18A900E582FAC4540FF582C00212188DD0E9
:0918B70002740F5AF58202188D2B
:0A18C000AA82782CE2F51908E2F57F
:0818CA001A08E2F51B08E2F523
:0718D2001C7830E2FF7B20CF
:0C18D900EF2FFFE51C235401FC4207E543
:0418E500192519F5B3
:0518E90019E51A33F5BA
:0518EE001AE51B33F5B3
:0518F3001BE51C33F5AC
:0518F8001CEFB5020029
:0918FD004007EFC39AFF431901F3
:09190600DBD1782CE519F208E5AB
:08190F001AF208E51BF208E5DD
:071917001CF27830EFF22210
:0C191E00AA82AB837827EAF208EBF2788B
:0A192A0033E2FA08E2FB08E2FC7861
:0A19340029EAF208EBF208ECF27861
:05193E0031E4F208F2A3
:0C1943007836E2FA08E2FB08E2FC8A8237
:0C194F008B838CF0121F5DFD7836740154
:0E195B002AF2E43B08F208ECF2EDFA70030207
:021969001F3B22
:05196B00BA2502800313
:03197000021F3320
:05197300C212C213C204
:0419780014C215C2BE
:04197C0016C217C2B6
:0419800018C21978F8
:0A1984003AE4F2783BE4F27DFF78CC
:09198E0036E2FE08E2FF08E2FB6C
:0E1997008E828F838BF0121F5DFAA3AE82AF9B
:0C19A500837836EEF208EFF208EBF2BA9D
:0919B10025078A8212185880896A
:0519BA008A04BC3000AE
:0919BF00403A8A047439B50400B1
:0C19C8004031BDFF22C006C007C00378FC
:0A19D4003BE275F00AA42A783B24D8
:0C19DE00D0F2D003D007D006783BE270B6
:0519EA00ACD21380A83F
:0C19EF00ED75F00AA4FC2A24D0FD809CB9
:0A19FB00BA2E07BDFF967D00809212
:051A05008A04BC610031
:091A0A0040108A04747AB504004E
:091A130040075302DFD2118002EA
:021A1C00C211F5
:051A1E00BA2002805512
:051A2300BA2B02804B0C
:051A2800BA2D0280410F
:051A2D00BA4202804BEB
:051A3200BA43028050E0
:061A3700BA4403021C1F6B
:061A3D00BA4603021C3D45
:061A4300BA4903021C1F5A
:051A4900BA4C028034DC
:061A4E00BA4F03021C2840
:061A5400BA5003021BAAB8
:051A5A00BA53028050A8
:061A5F00BA5503021C2F22
:061A6500BA5803021C3612
:031A6B00021C4119
:051A6E00D212021997DD
:051A7300D214021997D6
:051A7800D215021997D0
:051A7D00D217021997C9
:051A8200D218021997C3
:091A870030170C7939E314F879E9
:061A900039F3860280110B
:0A1A96007939E324FEF87939F3866C
:071AA00003088606188B0203
:081AA7008A82121858021C4C3F
:0A1AAF007939E324FDF87939F38654
:0C1AB900030886060886071818782CEB36
:0E1AC500F208EEF208EFF28B828E838FF0C0F3
:0E1AD30005121F45AB82AE83D005BDFF028B0E
:011AE10005FF
:0A1AE200201237783BC3E2F5F0EB69
:0B1AEC0095F0502C783BE2C39BF27891
:031AF7003BE2FED1
:0C1AFA008E071E783BEEF2EF6014758240
:0E1B060020C003C005C006121858D006D00536
:041B1400D00380E298
:041B1800783BEEF236
:0C1B1C00C003782CE2FE08E2FF08E2FBA8
:0E1B28008E828F838BF0121F5DFEFAD003EECB
:0E1B3600603B8D061DC374808EF063F08095B9
:0E1B4400F0502CC0038A82C003C0051218584E
:0C1B5200D005D003782CE2FE08E2FF086A
:071B5E00E2FB0EBE00010FC7
:0C1B6500782CEEF208EFF208EBF2D0034F
:021B710080A949
:061B7300201203021C4CCD
:0C1B7900783BC3E2F5F0EB95F04003026E
:021B85001C4CF6
:0A1B8700783BE2C39BF2783BE2FDDD
:0B1B91008D061D783BEDF2EE700302A4
:021B9C001C48E3
:0C1B9E00758220C005121858D00580E7A1
:0A1BAA007939E324FDF87939F38658
:0C1BB400060886070886041818782CEE36
:0C1BC000F208EFF208ECF2782EE2FABA1C
:021BCC00800097
:061BCE0040047A4380147C
:031BD400BA6000F4
:061BD70040047A50800B6F
:031BDD00BA40000B
:061BE00040047A49800276
:021BE6007A582B
:0E1BE8008A82C00212185875823A1218587577
:0E1BF6008230121858758278121858D002BA30
:041C04004902800D04
:051C0800BA5002800843
:081C0D00782DE2F5821218A9FE
:0A1C1500782CE2F5821218A9802D48
:091C1F00D216783A740AF280240E
:071C2800783A7408F2801DF8
:071C2F00783A740AF28016F6
:071C3600783A7410F2800FF0
:041C3D00D219800B2D
:071C41008A8212185880048A
:041C4800783BEDF206
:0A1C4C003019717939E324FCF879AE
:061C560039F38614088634
:061C5C001508861608863B
:071C620017181818782CE593
:081C690014F208E515F208E58C
:071C710016F208E517F278F6
:061C78002C7492F20874C6
:061C7E0020F2087480F260
:081C8400782CE2F51408E2F5EA
:081C8C001508E2F516740125AC
:071C940014FDE43515FEAF5D
:0A1C9B0016782CEDF208EEF208EFC7
:081CA500F28514828515838588
:0A1CAD0016F0121F5DFDFA7003022D
:021CB7001943CF
:071CB9008A8212185880C452
:081CC000783AE27003021943B7
:081CC8007A4230174AC002798C
:0A1CD00039E314F87939F3E6FE3326
:0C1CDA0095E0FFFDFC782CEEF208EFF224
:0C1CE60008EDF208ECF2D0023016030208
:021CF2001D8D46
:0C1CF400C002782CE2FC08E208E208E2E2
:0C1D00007E007F007D00782CECF208EEE5
:0B1D0C00F208EFF208EDF2D002807642
:0A1D170030182AC0027939E324FCD9
:0C1D2100F87939F3860408860608860766
:0C1D2D00088605181818782CECF208EE57
:0B1D3900F208EFF208EDF2D002804942
:0A1D4400C0027939E324FEF8793972
:0E1D4E00F3860408860618EE3395E0FFFD7854
:0C1D5C002CECF208EEF208EFF208EDF2B9
:0A1D6800D002201620C002782CE201
:0D1D7200FC08E2FE08E208E27F007D007838
:0C1D7F002CECF208EEF208EFF208EDF296
:021D8B00D00284
:0A1D8D0030162E782CE2FC08E2FE6E
:0E1D970008E2FF08E2FD30E71CC3E49CFCE418
:0C1DA5009EFEE49FFFE49DFD782CECF214
:0B1DB10008EEF208EFF208EDF28002ED
:021DBC00C2164D
:081DBE00D21A8A00793CE4F31B
:0A1DC6007930E4F3793AE3F582C0C6
:0A1DD000001218C0D000201A0E798E
:0C1DDA0030E3C4FDE2FE4DF218880280E8
:011DE60005F7
:051DE7007930E3FDF27C
:0A1DEC00793CE32401F3793CE3FBAA
:0A1DF600B21A792CE3FD09E3FE099F
:0E1E0000E3FF09E3FCED4E4F4C70BB88027807
:091E0E003CE2FB783BE270057830
:041E17003B7401F225
:0A1E1B0020132D20122AEB04FC789E
:031E25003BE2FDA0
:041E2800ECB5050010
:0E1E2C005019758220C002C003C004C0051208
:0D1E3A001858D005D004D003D0021D80E15F
:041E4700783BEDF205
:0B1E4B0030161575822DC002C0031276
:0C1E56001858D003D002783BE214F28050
:011E6200314E
:0C1E6300EB602E30141575822BC002C0FD
:0C1E6F0003121858D003D002783BE21494
:031E7B00F28016DC
:0B1E7E00301513758220C002C0031253
:0B1E89001858D003D002783BE214F29E
:071E940020122D783BE2FC57
:0B1E9B008C051C783BECF2EBB5050059
:091EA60050353013047D30800238
:021EAF007D2094
:0E1EB1008D82C002C003C004121858D004D0A5
:051EBF0003D00280D7F2
:0C1EC400783BC3E2F5F0EB95F050087895
:071ED0003BE2C39BF2800A14
:061ED700783BE4F28004F8
:041EDD00783BECF270
:021EE1008A0075
:0A1EE3008B041BEC602BB21A201ACE
:0C1EED000B08E2C4540FFC7930F38009AC
:091EF900E2FC53040F7930ECF314
:0C1F02007930E3F582C003C00012188D96
:061F0E00D000D00380CFDB
:061F140020120302194334
:041F1A00783BE2FB33
:091F1E008B041BEC700302194353
:0C1F2700758220C003121858D00380EB14
:081F33008A82121858021943BA
:0A1F3B007831E2F58208E2F5832216
:0B2092003C4E4F20464C4F41543E0096
:041F4500AA82AB833E
:081F4900121F5D6003A380F884
:0C1F5100C3E5829AF582E5839BF58322AC
:03048D0075812452
:0A049000121F8CE58260030204864F
:0E1F5D0020F71430F6148883A88220F507E6DA
:061F6B00A883758300222B
:031F7100E280F714
:031F7400E49322D1
:021F7700E02266
:0C1F79009003E0E493FA9003E1E4937815
:071F850009F28A82020C5AE6
:041F8C007582002238
:0B1F900000000000021F9B000000008A
:041F9B000000000042
:081F9F00E5826003D582EA220D
:00000001FF
